:1000000000EE00F010EE05F00CEC00F0000EF86EC3
:10001000060EF76EF3EF04F0EE6AE550E150FCE1F6
:06002000E250FAE11200BB
:1006000000414443205465737400000000EE00F084
:1006100011EE0CF0050EEECFE6FFE82EFCD7040E2F
:10062000010101010A6F000E01010B6F000E0101B3
:100630000101086F000E0101096F31D001010C0E9C
:10064000010101010A25E96EEA6A0101010EEA22AF
:100650000A0E01010101156F000E0101166F04C1A0
:1006600013F105C114F16FEC04F001010101135104
:10067000EF6E0A0E01010101156F000E0101166FE8
:1006800004C113F105C114F1D7EC03F013C104F157
:1006900014C105F1010101010A07D8A00B070101EE
:1006A000010105510411D8A401D001D0C7D701011F
:1006B00001010629D8B40729D8A401D001D015D04A
:1006C00004D001010101084B092B01010C0E0101AD
:1006D00001010825E96EEA6A0101010EEA22EF50E4
:1006E000D8B401D001D0EDD70FD0010101010651DE
:1006F000050801010101086F010101010751D8A09E
:10070000E82A00080101096F0101010105AF01D0CC
:1007100001D012D00101116F010E01010101146F0E
:10072000010111510101126F2D0E01010101136F21
:1007300001011251E2EC05F008C10AF109C10BF107
:10074000010101010B51800A800F050ED8B40A5D2A
:10075000D8A001D001D001D029D00101116F010E24
:1007600001010101146F0101115101010C0E010180
:1007700001010A25E96EEA6A0101010EEA22EF5041
:10078000300F01010101136FE2EC05F001010101DD
:100790000A4B0B2B010101010B51800A800F050E42
:1007A000D8B40A5DD8A001D001D0D7D7120001017A
:1007B0001B6F000E01010101186F01011B510101A6
:1007C000010116AF01D001D00FD001010101156D5B
:1007D0000101161FD8B0162B01011B6F010E01017C
:1007E0000101186F01011B510101010114AF01D07A
:1007F00001D00BD001010101136D0101141FD8B00C
:10080000142B010E01010101181B000E0101010151
:10081000196F000E01011A6F010101011651151126
:10082000D8B401D001D047D001011B6F010E0101E6
:100830000101176F01011B5109D00101D89001017D
:1008400015370101163701010101172B01010101C3
:1008500016AF01D001D0F1D70101D89001011937AD
:1008600001011A3701010101155101010101135D57
:10087000010101011651010101011459D8A001D053
:1008800001D00FD001010101155101010101135FD8
:1008900001010101165101010101145B0101010176
:1008A00019810101D89001011633010115330101AD
:1008B0000101172FD1D7010101011851D8B401D07E
:1008C00001D007D001010101196D01011A1FD8B033
:1008D0001A2B19C113F11AC114F100D01200010131
:1008E000196F000E01010101176F0101195101017A
:1008F000010114AF01D001D00FD001010101136D2E
:100900000101141FD8B0142B0101196F010E010150
:100910000101176F010119510101010116AF01D049
:1009200001D007D001010101156D0101161FD8B0DA
:10093000162B0101010116511511D8B401D001D0B7
:100940003ED00101196F010E01010101186F010173
:10095000195109D00101D89001011537010116374D
:1009600001010101182B0101010116AF01D001D0D5
:10097000F1D701010101155101010101135D0101CF
:1009800001011651010101011459D8A001D001D073
:100990000CD001010101155101010101135F010199
:1009A0000101165101010101145B0101D8900101FF
:1009B00016330101153301010101182FDAD70101A6
:1009C00001011751D8B401D001D007D001010101B4
:1009D000136D0101141FD8B0142B13C113F114C1EE
:1009E00014F100D01200640E01010101046F000E29
:1009F0000101056F8EEC06F00101026F010E01018D
:100A00000101046F01010251A0EC05F0A1EC06F018
:100A10000101026F000E01010101146F0101025179
:100A20000101036F010E01010101136F0101035167
:100A3000E2EC05F0010E01010101046F060E010157
:100A4000056F21EC06F00101026F000E01010101AA
:100A5000046F0101025148EC06F004C100F105C128
:100A600001F10101026F010E01010101056F010198
:100A700002510101036F000E01010101046F010128
:100A800003516DEC06F0040E01010101066F000E2A
:100A90000101076F00C104F101C105F106EC03F08B
:100AA000E80E01010101046F030E0101056F8EECD8
:100AB00006F0C9D700EF00F001011B6F000E010125
:100AC00001011A6F01011B510F0E95128A848A923F
:100AD00000D08C8800D083CF1AF1010101011A39AE
:100AE000F00B010101011A6F00D08C9800F000D0CA
:100AF00000D08C8800D083CF19F10F0E01010101C5
:100B00001917010101011A51010101011911010116
:100B100001011A6F010101011A51800B010101014C
:100B2000186F00D08C9800F000D000D001010101B6
:100B3000186701D001D0CDD78A94F00E9516120017
:100B4000C30E0101056F8E0EE82EFED7052FFCD7D0
:100B5000F00E9516959893929394F00E8C168C98AF
:100B60008A948A9200F08C888C8200F000D000D0A9
:100B70008C9800F000D000D05CEC05F00101056F0E
:100B8000000E01010101146F010105510101010174
:100B900004510C0901010101136FE2EC05F00101A0
:100BA000056F000E01010101146F010105510101E2
:100BB000066F280E01010101136F01010651E2ECDD
:100BC00005F012000101010113390F0B01010101B0
:100BD000156F0101010113510F0B01010101166F86
:100BE00001010101146701D001D002D08A9201D025
:100BF0008A8200D08C888C50F00B01010101151104
:100C000001010101176F17C18CFF00F000D000D067
:100C10008C9800F000D000D08C888C50F00B010133
:100C20000101161101010101176F17C18CFF00F0BE
:100C300000D000D08C9800F000D000D05CEC05F023
:100C4000120018D00101066F010E01010101146F9D
:100C500001010651010104C1F6FF010105C1F7FFC1
:100C600008000101F5CF13F1E2EC05F001010101EB
:100C7000044B052B010104C1F6FF010105C1F7FF7B
:100C80000800F5500009D8A401D001D0DBD712002C
:100C90000D0E01010101046501D001D008D0000E44
:100CA00001010101046F000E0101056F15D0000E56
:100CB000C26E010101010445E846FC0BC26EC28010
:100CC000C28200D0C2B201D001D0FCD7C290C3CF43
:100CD00004F1C4CF05F100D01200280E010101017A
:100CE000046101D001D019D0010101010551D8B42E
:100CF00001D001D003D001010101048D01010101E6
:100D0000048F0101066F000E01010101146F010142
:100D1000065104C113F1E2EC05F0120009D0A60E51
:100D2000E82EFED700D0010101010407D8A0050775
:100D30000101010105510411D8A401D001D0EFD760
:100D400012000101046F8A0EC06E010104511200ED
:020000040030CA
:0A00000000021F1E0081C1000FC0A6
:00000001FF
